:1000000049288F018E00FF308E07031C8F07031CC9
:10001000442803308D00DF300F2003288D01E83E97
:100020008C008D09FC30031C18288C070318152838
:100030008C0764008D0F15280C181E288C1C222894
:100040000000222808008D018F018E0002302D282B
:100050008D018F018E0004302D2894000F080D02B1
:10006000031D34280E080C02043003180130031954
:1000700002301405031DFF3044280038031DFF30F3
:100080000405031DFF304428831303138312640007
:1000900008008316F830850086018312FF30860041
:1000A0007B28051A2B15051E2B11A9010030051AF6
:1000B00001308C0000302B19013023209E002908CC
:1000C0008C0032302820A0001E08840020083D202B
:1000D000A000A10064002008210403197128A90AC6
:1000E000562864002908323C0319992A04308D00EF
:1000F0004C300F200800A9016400051E80287C28D0
:100100000030051A01308C00003023209E002908A1
:100110008C0034302820A0001E08840020083D20D8
:10012000A000A10064002008210403199928A90A4D
:10013000802801308D00F4300F20512003012B194D
:100140000130013A03192813031D281751202B19D8
:10015000AB152B1DAB1151202B1928162B1D281266
:1001600051202B19A8152B1DA81151202B1928152A
:100170002B1D281151202B19A8142B1DA81051201C
:100180002B1928142B1D281051202B19AA162B1DB2
:10019000AA1251202B192A162B1D2A1251202B1975
:1001A000AA152B1DAA1151202B192A152B1D2A1116
:1001B00051202B19AA142B1DAA1051202B192A14D7
:1001C0002B1D2A1064000301AB19013E2B18013CC2
:1001D000031DEB287F2AAB192B14AB1D2B102A080B
:1001E0008C00013023209E000030061801308C0066
:1001F00000302320A0001E08840020083D20A0001D
:10020000A1006400200821040319082906147F2A8C
:100210002A088C00013023209E000030061801308F
:100220008C0001302320A0001E08840020083D20FF
:10023000A000A10064002008210403192129061050
:100240007F2A2A088C00023023209E000030861866
:1002500001308C0000302320A0001E0884002008FC
:100260003D20A000A10064002008210403193A29C0
:1002700086147F2A2A088C00023023209E0000303A
:10028000861801308C0001302320A0001E08840055
:1002900020083D20A000A1006400200821040319CB
:1002A000532986107F2A2A088C00033023209E00C1
:1002B0000030061901308C0000302320A0001E08F9
:1002C000840020083D20A000A10064002008210433
:1002D00003196C2906157F2A2A088C000330232075
:1002E0009E000030061901308C0001302320A00050
:1002F0001E08840020083D20A000A1006400200802
:1003000021040319852906117F2A2A088C0004304C
:1003100023209E000030861901308C0000302320FD
:10032000A0001E08840020083D20A000A100640059
:100330002008210403199E2986157F2A2A088C008B
:10034000043023209E000030861901308C000130DB
:100350002320A0001E08840020083D20A000A1004A
:100360006400200821040319B72986117F2A2A086E
:100370008C00053023209E000030061A01308C00CE
:1003800000302320A0001E08840020083D20A0008B
:10039000A1006400200821040319D02906167F2A31
:1003A0002A088C00053023209E000030061A0130F8
:1003B0008C0001302320A0001E08840020083D206E
:1003C000A000A1006400200821040319E9290612F5
:1003D0007F2A2A088C00063023209E000030861ACF
:1003E00001308C0000302320A0001E08840020086B
:1003F0003D20A000A1006400200821040319022A66
:1004000086167F2A2A088C00063023209E000030A2
:10041000861A01308C0001302320A0001E088400C1
:1004200020083D20A000A100640020082104031939
:100430001B2A86127F2A2A088C00073023209E0060
:100440000030061B01308C0000302320A0001E0865
:10045000840020083D20A000A100640020082104A1
:100460000319342A06177F2A2A088C000730232014
:100470009E000030061B01308C0001302320A000BC
:100480001E08840020083D20A000A1006400200870
:10049000210403194D2A06137F2A2A088C000830EC
:1004A00023209E000030861B01308C00003023206A
:1004B000A0001E08840020083D20A000A1006400C8
:1004C000200821040319662A86177F2A2A088C002F
:1004D000083023209E000030861B01308C00013044
:1004E0002320A0001E08840020083D20A000A100B9
:1004F00064002008210403197F2A86137F2AAB1980
:100500008515AB1D85117B28051401308F00F43053
:100510000220051001308F00F43002200514013054
:100520008F00F4300220051001308F00F4300220DB
:100530007B28051401308F00F430022005100130B3
:100540008F00F4300220051401308F00F4300220B7
:0C055000051001308F00F43002207B28E1
:02400E00F53F7C
:00000001FF
